:20F800000F120F43D2B323001C24D2B320001920D2B324001624D2C32300E2B3200011202E
:20F82000D2C325001F43F2F0CF002300F2F0CF002500E2D32400E2C32300E2D32500D24372
:20F840000002E2B323001324E2B320001020E2B324000D24E2C32300E2C325001F43E2C34F
:20F860002400E2C32300E2D32500D2430102E2B323002F24E2B320002C24E2B32400292098
:20F88000E2C32300E2C325001F43C29301022124E2D22200F2C221000D123D4086051D8365
:20F8A000FE233D410343E2C221000D123D4086051D83FE233D410343E2D221000D123D4081
:20F8C00054371D83FE233D410343F2D22100E2C22200F2B0100023002424F2B0100020007E
:20F8E0002020F2B0100024001C24F2F0EF002300F2B0200020001520F2F0EF0025001F434F
:20F90000F2F0FC002300F2F0FC002500F2D020002400F2F0DF002300F2D020002500D243DD
:20F920000002F2B0200023001A24F2B0200020001620F2B0200024001224F2F0DF0023008A
:20F94000F2F0DF0025001F43F2F0DF002400F2F0DF002300F2D020002500D2430102F2B0D5
:20F96000200023003824F2B0200020003424F2B0200024003020F2F0DF002300F2F0DF00D3
:20F9800025001F43C29301022624F2D040002200F2F07F0021000D123D408B001D83FE23B0
:20F9A0003D410343F2F0BF0021000D123D4086051D83FE233D410343F2D0400021000D12D3
:20F9C0003D400F0B1D83FE233D41F2D080002100F2F0BF0022000F930720F2F0CC0025008F
:20F9E000D2430002C2432300B2404B007201B24010006201B24016016001B1C0F8000200DE
:20FA00003F410013B240805A2001F2F0F8005700F2D00B005700F2D0B0005700F2D0200066
:20FA20005300E2B302000A24E2C302003F40FF0F1F93F73B1F831F93F43BFC3FB2401000D6
:20FA40006401B240EE027401B2402601600132D0D800F2F0FC002200E2C22200F2D22200EA
:20FA6000F2D22100F2F0CF002200F2F0BF002200F2D080002200F2D080002100D2C323008C
:20FA8000D2D32400D2D32500F2F0EF002300F2D010002400F2D010002500023C32D0F800BA
:20FAA000C2930002FB2732D0D800FA3F0A1209123F4000003F90000004243C400000B012CF
:20FAC0007EFB3F40CCFC3F90D0FC16243F40D0FC3F90D4FC11243A40D4FC3A80D0FC0A1187
:20FAE0000A113940D0FC3C497F4C0F5F1F4FCCFC3D498F121A83F723B012C4FC3F400000D3
:20FB00003F90000008243A400000023C3F4A8F123A900000FB233040A6FC0A1209127A4C11
:20FB2000213C1C530E930D243F9000010A2C29434F4F8F107B4C0FDB1983FA23023C2F920F
:20FB400002287B4C013C0B4A1F833F930B244B4B1D53CD4BFFFF1F833F93FA23033C1D5323
:20FB6000CD4FFFFF7F4C0F9AFA237F4C0F93E7237F4C8F106B4C0F5BD4233040A6FC0A12B3
:20FB80000912094C1B4902000A43223C0C4A3D400600B01264FC0C591E4C08001D4C0400A5
:20FBA0001F4C06000C4F0E930E203E40CCFC3E90D0FC0D246E4D0E5E1E4ECCFC1D530C4D75
:20FBC0000D4F8E12023CB0128AFC1B4902001A530A9BDC2B3040A6FC82436001B2F0EFFF5C
:20FBE0006201C2430002C2430102F2D00C002100E2C22200D2D32400F2F0FC002300E2C36F
:20FC00002500D2D32500F2D0C0002100F2F0BF002200F2D010002400F2F0CF002300F2F0E3
:20FC2000DF002500F2D010002500B1C0D8000000001331407E02B012C0FC0C930224B01277
:20FC4000ACFA0C43B01204FAB012B4FCA2932E01052082436001B2F0EFFF6401B1C0D80090
:20FC6000000000130E4312C30C1001280E5D0D5D0C93F9230C4E30410F4C0C4D3D40030077
:20FC80000D5F1E4F010030408AFC0F4C0E9305241F53FF4DFFFF1E83FB2330413441354198
:20FCA00036413741384139413A41304132D01000FD3F03430343FF3F03431E4330401AFB32
:06FCC0001C4330413041FD
:0EFCC600010002000000BAFC78FCC6FC00023F
:02FFE40000F823
:02FFE600ACFC71
:02FFE800ACFC6F
:02FFF0004CFCC7
:02FFF200D8FB3A
:02FFF400ACFC63
:02FFFC00ACFC5B
:02FFFE0032FCD3
:00000001FF
